:020000040000FA
:020000000528D1
:08000800532903138312850143
:1000100007309F008316203085000130860081154F
:1000200081128312A901AA01A201A301A401A501C1
:10003000A6011330A0008830A1002A1444308100AA
:10004000A0308B00AB010330AC20A9193628291E43
:100050002E2802302C0203192912222806183628CD
:100060002B1834282B142328412022282B10851EDE
:100070003B28A9112228AB183F28AB14232879204C
:100080002228AC010330AC20061C4A282B1C772800
:100090002B1042282B1402302C02031D4228291455
:1000A000AC01AD016430AE000330AC20851E5E288B
:1000B000061C60282B1C6F282B1054283221622824
:1000C00012212B142E082B1DC830AC202B15AD018E
:1000D00005302C02031D54280A30AE0054282B1181
:1000E000AC016430AE0005302D02031D54282910E8
:1000F00008002408031D802806302302031C8B28D7
:1001000005302402031D982805302302031C98287B
:100110008B131F218C288B13A201A301A401133080
:10012000A0008830A100443081002A148B17A02839
:10013000A9150618A0280230A906A9112916AC0194
:10014000080082078034F234483460343234243476
:100150000434F03400342034AF00FE30860005143F
:10016000A91CB5282608A120C028E7202808031DBF
:10017000BB28FE30BC28A120291DBE392919DE3933
:10018000860085114E21FE3086008515A91C2708A2
:10019000A9182508A120860005112A1805124E214C
:1001A0000516FE30860005152408A120860085105E
:1001B0004E21FE30860085142308A12086000510FC
:1001C000291805124E210516AF0BAD280800250889
:1001D000A7002608A800031DF4282708031D0E29E0
:1001E000A80A0230A7000E2901302802031D0229A7
:1001F0000230270203191029031C0E29A80102301E
:10020000A70210290230270203180A29A801083082
:10021000A7071029A8030230A702102929111129C4
:1002200029150800A201A30A0A302302031D31295F
:10023000A301A40A06302402031D3129A401A50A42
:100240000430250203192B290A302502031D312908
:10025000A501A60A312902302602031D3129A50174
:10026000A6010800A2010130A30203184D2909309C
:10027000A3000130A40203184D290530A400013069
:10028000A50203184D290930A5000130A602031864
:100290004D290230A6000330A50008006430B000EC
:1002A000B00B50290800F0000308F100831244301D
:1002B00081000B110130A102031CA00309302002B0
:1002C000031D6829C4302102031D68292A109929B9
:1002D000A008031D9929A108031D99292A14AC0A15
:1002E000AD0AA20A3C302202031D9529A201A30AED
:1002F0000A302302031D9529A301A40A0630240213
:10030000031D9529A401A50A0430250203198F298C
:100310000A302502031D9529A501A60A9529023058
:100320002602031D9529A501A6011330A0008830DF
:0C033000A10071088300F00E700E09009F
:02400E00023F6F
:00000001FF
